:020000040000FA
:040000003CEF01F0E0
:080008003AEF01F048414E53AC
:100010002050554E43482072657631382A2A2A4DA1
:1000200041494E204D454E552A2A2A20312E4D4118
:100030004E55414C206D6F76696E6720322E5245C9
:100040004144204D4944492066696C65332E4E4F2A
:10005000524D414C2053544152542020342E52458D
:1000600053544152542066726F6D2020352E5055E6
:100070004E4348202073657474696E67362E4E4F68
:10008000544520706F736974696F6E20372E424F2C
:100090004F4B20737065656420736574382E436C14
:1000A000454152206E6F746520736574392E41523C
:1000B0004D20494E495420202020202031302E53FD
:1000C00041564520546F6E652073657431312E4C56
:1000D0004F414420546F6E652073657431322E5445
:1000E00045535420202020202020202041726D20C4
:1000F00020737470426F6F6B2073747050756E63F1
:100100002020777450756E632053544B50756E6386
:100110002044494141726D20636F7272426F6F6B70
:1001200020636F724D61782064657620696E206D62
:100130006D2F733A436C656172696E674E65772007
:1001400066696C6553707572202020202020202065
:100150002020202041726D20696E69744E43205327
:10016000544F502041726D20696E69744445562089
:10017000484947485345542041524D215354415218
:10018000543F202052454144494E472020484F4C7F
:100190004420202046494C452065727208500A02CE
:1001A000F3500E6EF4500F6E106A116A08500B0275
:1001B000F3500F26F4501022000E086E1122085042
:1001C0000C02F3501026F450112208500D02F35087
:1001D000112609500A02F3500F26F4501022000E87
:1001E000086E112209500B02F3501026F450112210
:1001F00009500C02F35011261200200E1A6E0C6AE0
:100200000D6A0E6A0F6AD8901436153616361736F0
:10021000D890083609360A360B360C360D360E36AF
:100220000F360F50135CD8A422EF01F00E50125C71
:10023000D8A422EF01F00D50115CD8A422EF01F0F8
:100240000C50105CD8B428EF01F0D8B036EF01F0B4
:10025000D8800C5010540C6E0D5011540D6E0E5071
:1002600012540E6E0F5013540F6E14801A2E03EF9B
:1002700001F01200DDEF0EF054EF01F002014B6FC0
:10028000F00E8C144C6F0F0E4B154D6F4C118C6E85
:1002900012000201486F0F0E8C14496F4839F00BA1
:1002A0004A6F49118C6E1200D190FC0ED3169B9CA4
:1002B000C26A0F0EC16EC06A070EB46E9692969413
:1002C000939093929394939640EF02F00201456FBE
:1002D0004551D8B412004505D8A478EF01F00001CB
:1002E0000A0E086E082E72EF01F0000000001200E6
:1002F00045070001070E086E082E7CEF01F0000094
:1003000002014551466F476B8EEF01F000010E0E62
:10031000086E082E89EF01F00201472B4751465D18
:10032000D8A486EF01F012003F51416F4051426F57
:10033000436B446BACEF01F00001090E086EB70E81
:10034000096E092EA1EF01F0082E9FEF01F00000C9
:100350000201432BD8B4442B4351415D086E4451F4
:10036000425D0810D8A49CEF01F0120039513B6F98
:100370003A513C6F3D6B3E6BD2EF01F00001110E24
:10038000086E570E096E6F0E0A6E0A2EC5EF01F049
:10039000092EC3EF01F0082EC1EF01F002013D2B41
:1003A000D8B43E2B3D513B5D086E3E513C5D08107C
:1003B000D8A4BEEF01F012003351356F3451366FBF
:1003C000376B386BF8EF01F000013D0E086ED60E6A
:1003D000096E7E0E0A6E0A2EEBEF01F0092EE9EF90
:1003E00001F0082EE7EF01F00201372BD8B4382BCB
:1003F0003751355D086E3851365D0810D8A4E4EFEA
:1004000001F012000201326F32B10AEF02F08A9657
:100410000BEF02F08A8632B311EF02F08A9412EFEA
:1004200002F08A8432B518EF02F08A9219EF02F0D6
:100430008A8232B71FEF02F08A9020EF02F08A80A2
:100440008D84000000000000000000008D94120068
:10045000306F30390F0B316F02EC02F00201305176
:1004600002EC02F0040E66EF01F02F6F8D822F5127
:1004700028EF02F002012E6F8D922E5128EF02F02C
:100480001C6AC0EF02F02D6F020E2D5DD8B44CEF48
:1004900002F0D8A04DEF02F02D6B2D51D8B4000C16
:1004A0002D05D8B4400C020E2D5DD8B4100C030EEF
:1004B0002D5DD8B4500C1200800E1C1002012C6F60
:1004C0003AEF02F002012B6F35EF02F002012A6FC2
:1004D00035EF02F00201276F43EC02F00201296FB1
:1004E000285129251C6E5CEF02F0010E3AEC02F057
:1004F000B40E66EF01F00201256F43EC02F01C6EB2
:100500005CEC02F00201266B200E66EC02F00201A8
:10051000262B100E265DD8A484EF02F05CEF02F0CB
:100520008D92190E02013F6F406B94EC01F0030EA7
:1005300002EC02F0050E02013F6F406B94EC01F0FB
:10054000030E02EC02F00A0E66EC01F0030E02EC60
:1005500002F0040E66EC01F0020E02EC02F0040E52
:1005600066EC01F0280E3AEC02F01C0E3AEC02F0B8
:100570000C0E3AEC02F0060E3AEC02F075EF02F0C7
:1005800090EC02F02DEF03F01E51216F1F51226FEE
:10059000236B246BA6B2CAEF02F02151A96EA69C70
:1005A000A69EA680A850206F12000201186F165157
:1005B0001A6F17511B6F1C6B1D6BA6B2DDEF02F09B
:1005C0001A51A96EA69CA69E1851A86EA6841991D0
:1005D000F2BE1981F29E550EA76EAA0EA76EA682D4
:1005E0000000000019B1F8EF02F0F29EF9EF02F0FE
:1005F000F28EA6941200B886AC849F0EAF6EB06ADD
:100600001200AC6AAB6AFBEC02F09D9A9D98948E46
:10061000948CAC8AAB8EAB8812000201156F9EA839
:100620000FEF03F01551AD6E12009EAA1EEF03F0FE
:10063000AE500201136F9E9A22EF03F00201149153
:1006400028EF03F0ABA227EF03F0AB98AB8814813F
:10065000089014B108801351120001EC03F06CEF04
:1006600003F00201126FC96EC6BEFF0CC7A036EFC1
:1006700003F0C95012000201116F31EF03F0FF0EB9
:1006800031EC03F00201106F12000E6FC66AC78EC4
:100690000E51D8A450EF03F0C698C78C63EF03F057
:1006A0000E05D8A458EF03F0C698C79C63EF03F07B
:1006B000020E0E5DD8A461EF03F0C688C78C63EF0D
:1006C00003F0C688C79C0F0E0F15086EF00EC614F7
:1006D0000810C66EC68A12009488949A94960201F5
:1006E0000F6B030E45EC03F0929A898A01EF04F038
:1006F000C698C78C0B6B000E0A5DD8A48CEF03F074
:10070000000E095DD8A48CEF03F0FF0E085DD8A49D
:100710008CEF03F0FF0E075DD8B494EF03F0D8A080
:1007200094EF03F0010E0B6F0851086E0951096E2A
:100730000A510A6E0B6A08500C6F07510D6F899AA7
:10074000050E3F6F406B94EC01F0020E3BEC03F0A2
:1007500002010B513BEC03F002010C513BEC03F0A6
:1007600002010D513BEF03F00201066F3BEF03F076
:10077000898A1200C698C78C0001FF6B000E020127
:10078000035DD8A4D0EF03F0000E025DD8A4D0EF33
:1007900003F0FF0E015DD8A4D0EF03F0FF0E005D63
:1007A000D8B4D9EF03F0D8A0D9EF03F0010E0001BF
:1007B000FF6F02010151086E0251096E03510A6E6A
:1007C0000B6A0850046F0051056F899A050E3F6F40
:1007D000406B94EC01F0030E3BEC03F00001FF5181
:1007E0003BEC03F0020104513BEC03F00201055124
:1007F0003BEF03F03FEC03F00001FE6F1200898A2B
:100800001200010E0201336F346BDCEC01F09680B4
:100810009284928092889282948092869482939815
:100820008A98948495909592959495969598959A92
:10083000959C959E000E3EEC01F0000E49EC01F0F7
:10084000010E1E6E010E1F6E010E226E236A010E36
:10085000266E276A286A296A0A0E346E0A0E356ED9
:10086000320E366E640E376E640E386E0A0E396EB6
:10087000640E3A6E3B6A460E3E6E3F6A1E0E406E36
:10088000320E416E426AF80ED5140109D56ED59A22
:10089000D596D59CF294F28AF28EF28C010E456EBA
:1008A000466A476A536AF1EF13F0FC6F0F0EFC17AC
:1008B000010EFD6FFC05D8A462EF04F0030EFC6F7F
:1008C000A2EF04F0030EFC5DD8A46DEF04F0060E59
:1008D000FC6F020EFD6FA2EF04F0020EFC5DD8A4C7
:1008E00076EF04F0060EFC6FA2EF04F0060EFC5D3E
:1008F000D8A481EF04F00C0EFC6F020EFD6FA2EF86
:1009000004F0040EFC5DD8A48AEF04F00C0EFC6F1A
:10091000A2EF04F00C0EFC5DD8A495EF04F0090ED4
:10092000FC6F020EFD6FA2EF04F0080EFC5DD8A470
:100930009EEF04F0090EFC6FA2EF04F0030EFC6FB3
:10094000020EFD6FFC511200FA6F0F0EFA17010E26
:10095000FB6F080EFA5DD8A4B2EF04F00C0EFA6F2C
:10096000F1EF04F00C0EFA5DD8A4BDEF04F0060E12
:10097000FA6F020EFB6FF1EF04F0040EFA5DD8A4DB
:10098000C6EF04F0060EFA6FF1EF04F0060EFA5D02
:10099000D8A4D1EF04F0030EFA6F020EFB6FF1EF53
:1009A00004F0020EFA5DD8A4DAEF04F0030EFA6F39
:1009B000F1EF04F0030EFA5DD8A4E5EF04F0090EA0
:1009C000FA6F020EFB6FF1EF04F0FA05D8A4EDEF19
:1009D00004F0090EFA6FF1EF04F00C0EFA6F020E3C
:1009E000FB6FFA5112000001F86F010EF96F0F0E44
:1009F000F817F805D8A401EF05F0030EF86F39EFEA
:100A000005F0030EF85DD8A40AEF05F0020EF86FAA
:100A100039EF05F0020EF85DD8A413EF05F0060ECD
:100A2000F86F39EF05F0060EF85DD8A41CEF05F05D
:100A3000040EF86F39EF05F0040EF85DD8A425EF29
:100A400005F00C0EF86F39EF05F00C0EF85DD8A428
:100A50002EEF05F0080EF86F39EF05F0080EF85D7F
:100A6000D8A437EF05F0090EF86F39EF05F0010E45
:100A7000F86FF85112000001F66F010EF76F0F0EBC
:100A8000F617080EF65DD8A44AEF05F00C0EF66FC7
:100A900081EF05F00C0EF65DD8A453EF05F0040EBF
:100AA000F66F81EF05F0040EF65DD8A45CEF05F05B
:100AB000060EF66F81EF05F0060EF65DD8A465EF21
:100AC00005F0020EF66F81EF05F0020EF65DD8A478
:100AD0006EEF05F0030EF66F81EF05F0030EF65D85
:100AE000D8A477EF05F0010EF66F81EF05F0F6055B
:100AF000D8A47FEF05F0090EF66F81EF05F0080E20
:100B0000F66FF65112001E50A4EC04F01E6E0001A8
:100B1000FB511D6E1E5049EC01F0345002013F6F35
:100B2000406B94EC01F0D88024501D540001F46F08
:100B3000000E086E25500854F56F2350F55DD8A4BB
:100B4000A4EF05F02250F45DD8B4AAEF05F0D8A0C8
:100B5000B0EF05F01D502226000E086E2322120071
:100B60002250246E2350256E12001E5055EC04F0C6
:100B70001E6E0001FD511D6E1E5049EC01F0245007
:100B80001D240001F26F000E086E25500820F36F3F
:100B90002350F35DD8A4CFEF05F02250F25DD8B416
:100BA000D5EF05F0D8B0E0EF05F0D88022501D5405
:100BB000226E000E086E23500854236EE4EF05F0F9
:100BC0002250246E2350256E345002013F6F406B3B
:100BD00094EF01F01F5055EC04F01F6E0001FD5121
:100BE0001D6E1F503EEC01F02A501D240001EE6FD7
:100BF000000E086E2B500820EF6F2C500820F06F6D
:100C00002D500820F16F2950F15DD8A414EF06F0A3
:100C10002850F05DD8A414EF06F02750EF5DD8A45B
:100C200014EF06F02650EE5DD8B41AEF06F0D8B0F7
:100C30002BEF06F0D88026501D54266E000E086E4D
:100C400027500854276E28500854286E29500854FD
:100C5000296E33EF06F026502A6E27502B6E28504F
:100C60002C6E29502D6E355002013F6F406B94EF72
:100C700001F01F50A4EC04F01F6E0001FB511D6E2B
:100C80001F503EEC01F0D8802A501D540001EA6F3D
:100C9000000E086E2B500854EB6F2C500854EC6F6C
:100CA0002D500854ED6F2950ED5DD8A464EF06F087
:100CB0002850EC5DD8A464EF06F02750EB5DD8A473
:100CC00064EF06F02650EA5DD8B46AEF06F0D8A0CB
:100CD00075EF06F01D502626000E086E27220850DC
:100CE0002822085029227DEF06F026502A6E275030
:100CF0002B6E28502C6E29502D6E355002013F6FFF
:100D0000406B94EF01F01E503BEC05F01E6E0001AD
:100D1000F7511D6E1E5049EC01F0D88024501D542F
:100D20000001E86F000E086E25500854E96F23504B
:100D3000E95DD8A49EEF06F02250E85DD8B4A4EF98
:100D400006F0D8A0ABEF06F01D502226000E086E6C
:100D50002322AFEF06F02250246E2350256E34502C
:100D600002013F6F406B94EF01F01E50F3EC04F072
:100D70001E6E0001F9511D6E1E5049EC01F0245009
:100D80001D240001E66F000E086E25500820E76F55
:100D90002350E75DD8A4CFEF06F02250E65DD8B42B
:100DA000D5EF06F0D8B0E0EF06F0D88022501D5401
:100DB000226E000E086E23500854236EE4EF06F0F6
:100DC0002250246E2350256E345002013F6F406B39
:100DD00094EF01F01F50F3EC04F01F6E0001F95185
:100DE0001D6E1F503EEC01F02A501D240001E26FE1
:100DF000000E086E2B500820E36F2C500820E46F83
:100E00002D500820E56F2950E55DD8A414EF07F0B8
:100E10002850E45DD8A414EF07F02750E35DD8A470
:100E200014EF07F02650E25DD8B41AEF07F0D8B0FF
:100E30002BEF07F0D88026501D54266E000E086E4A
:100E400027500854276E28500854286E29500854FB
:100E5000296E33EF07F026502A6E27502B6E28504C
:100E60002C6E29502D6E355002013F6F406B94EF70
:100E700001F01F503BEC05F01F6E0001F7511D6E95
:100E80001F503EEC01F0D8802A501D540001DE6F47
:100E9000000E086E2B500854DF6F2C500854E06F82
:100EA0002D500854E16F2950E15DD8A464EF07F09C
:100EB0002850E05DD8A464EF07F02750DF5DD8A488
:100EC00064EF07F02650DE5DD8B46AEF07F0D8A0D3
:100ED00075EF07F01D502626000E086E27220850D9
:100EE0002822085029227DEF07F026502A6E27502D
:100EF0002B6E28502C6E29502D6E355002013F6FFD
:100F0000406B94EF01F0DB6F0201286B0001DC51B4
:100F10006AEC02F00001DD6BDD6BDB51D8A4A2EFBF
:100F200007F01C0EF66E000EF76E000EF86EDD5127
:100F3000F626000E086EF7220850F8220900F55038
:100F400062EC02F00001DB05D8A4B8EF07F02C0E2C
:100F5000F66E000EF76E000EF86EDD51F626000EEE
:100F6000086EF7220850F8220900F55062EC02F0F2
:100F7000020E0001DB5DD8A4CFEF07F03C0EF66E49
:100F8000000EF76E000EF86EDD51F626000E086EAC
:100F9000F7220850F8220900F55062EC02F0030E27
:100FA0000001DB5DD8A4E6EF07F04C0EF66E000EF4
:100FB000F76E000EF86EDD51F626000E086EF72271
:100FC0000850F8220900F55062EC02F0040E00010E
:100FD000DB5DD8A4FDEF07F05C0EF66E000EF76E39
:100FE000000EF86EDD51F626000E086EF72208504E
:100FF000F8220900F55062EC02F0050E0001DB5DFD
:10100000D8A414EF08F06C0EF66E000EF76E000E0A
:10101000F86EDD51F626000E086EF7220850F82211
:101020000900F55062EC02F0060E0001DB5DD8A469
:101030002BEF08F07C0EF66E000EF76E000EF86EC9
:10104000DD51F626000E086EF7220850F82209003E
:10105000F55062EC02F0070E0001DB5DD8A442EF10
:1010600008F08C0EF66E000EF76E000EF86EDD5175
:10107000F626000E086EF7220850F8220900F550F7
:1010800062EC02F0080E0001DB5DD8A459EF08F015
:101090009C0EF66E000EF76E000EF86EDD51F62611
:1010A000000E086EF7220850F8220900F55062EC95
:1010B00002F0090E0001DB5DD8A470EF08F0AC0E61
:1010C000F66E000EF76E000EF86EDD51F626000E7D
:1010D000086EF7220850F8220900F55062EC02F081
:1010E0000A0E0001DB5DD8A487EF08F0BC0EF66E97
:1010F000000EF76E000EF86EDD51F626000E086E3B
:10110000F7220850F8220900F55062EC02F00B0EAD
:101110000001DB5DD8A49EEF08F0CC0EF66E000E49
:10112000F76E000EF86EDD51F626000E086EF722FF
:101130000850F8220900F55062EC02F00C0E000194
:10114000DB5DD8A4B5EF08F0DC0EF66E000EF76E8E
:10115000000EF86EDD51F626000E086EF7220850DC
:10116000F8220900F55062EC02F0140E0001DB5D7C
:10117000D8A4CCEF08F00C0EF66E000EF76E000E41
:10118000F86EDD51F626000E086EF7220850F822A0
:101190000900F55062EC02F00001DD2B100EDD5D60
:1011A000D8A48DEF07F012000001D96F140ED95D9D
:1011B000D8B4E6EF08F0D8B0E6EF08F0010E02016F
:1011C000286F010E6AEC02F0ECEF08F0080E020145
:1011D000286F010E6AEC02F00001DA6BDA6BD905B8
:1011E000D8A404EF09F0EC0EF66E000EF76E000EB8
:1011F000F86EDA51F626000E086EF7220850F82233
:101200000900F55062EC02F0020E0001D95DD8A48D
:101210001BEF09F0F40EF66E000EF76E000EF86E7E
:10122000DA51F626000E086EF7220850F82209005F
:10123000F55062EC02F0030E0001D95DD8A432EF44
:1012400009F0FC0EF66E000EF76E000EF86EDA5125
:10125000F626000E086EF7220850F8220900F55015
:1012600062EC02F0040E0001D95DD8A449EF09F048
:10127000040EF66E010EF76E000EF86EDA51F626C9
:10128000000E086EF7220850F8220900F55062ECB3
:1012900002F0050E0001D95DD8A460EF09F00C0E34
:1012A000F66E010EF76E000EF86EDA51F626000E9D
:1012B000086EF7220850F8220900F55062EC02F09F
:1012C000060E0001D95DD8A477EF09F0140EF66E72
:1012D000010EF76E000EF86EDA51F626000E086E5B
:1012E000F7220850F8220900F55062EC02F0070ED0
:1012F0000001D95DD8A48EEF09F01C0EF66E010E28
:10130000F76E000EF86EDA51F626000E086EF72220
:101310000850F8220900F55062EC02F0080E0001B6
:10132000D95DD8A4A5EF09F0240EF66E010EF76E74
:10133000000EF86EDA51F626000E086EF7220850FD
:10134000F8220900F55062EC02F0090E0001D95DA7
:10135000D8A4BCEF09F02C0EF66E010EF76E000E4D
:10136000F86EDA51F626000E086EF7220850F822C1
:101370000900F55062EC02F00A0E0001D95DD8A414
:10138000D3EF09F0340EF66E010EF76E000EF86E14
:10139000DA51F626000E086EF7220850F8220900EE
:1013A000F55062EC02F00B0E0001D95DD8A4EAEF13
:1013B00009F03C0EF66E010EF76E000EF86EDA5173
:1013C000F626000E086EF7220850F8220900F550A4
:1013D00062EC02F00C0E0001D95DD8A401EF0AF016
:1013E000440EF66E010EF76E000EF86EDA51F62618
:1013F000000E086EF7220850F8220900F55062EC42
:1014000002F0140E0001D95DD8A418EF0AF04C0EBA
:10141000F66E010EF76E000EF86EDA51F626000E2B
:10142000086EF7220850F8220900F55062EC02F02D
:10143000150E0001D95DD8A42FEF0AF0540EF66EF8
:10144000010EF76E000EF86EDA51F626000E086EE9
:10145000F7220850F8220900F55062EC02F0160E4F
:101460000001D95DD8A446EF0AF05C0EF66E010EBD
:10147000F76E000EF86EDA51F626000E086EF722AF
:101480000850F8220900F55062EC02F0170E000136
:10149000D95DD8A45DEF0AF0640EF66E010EF76E0A
:1014A000000EF86EDA51F626000E086EF72208508C
:1014B000F8220900F55062EC02F0180E0001D95D27
:1014C000D8A474EF0AF06C0EF66E010EF76E000EE3
:1014D000F86EDA51F626000E086EF7220850F82250
:1014E0000900F55062EC02F0190E0001D95DD8A494
:1014F0008BEF0AF0740EF66E010EF76E000EF86EAA
:10150000DA51F626000E086EF7220850F82209007C
:10151000F55062EC02F01A0E0001D95DD8A4A2EFDA
:101520000AF07C0EF66E010EF76E000EF86EDA51C0
:10153000F626000E086EF7220850F8220900F55032
:1015400062EC02F01B0E0001D95DD8A4B9EF0AF0DD
:10155000840EF66E010EF76E000EF86EDA51F62666
:10156000000E086EF7220850F8220900F55062ECD0
:1015700002F01C0E0001D95DD8A4D0EF0AF08C0E49
:10158000F66E010EF76E000EF86EDA51F626000EBA
:10159000086EF7220850F8220900F55062EC02F0BC
:1015A0001D0E0001D95DD8A4E7EF0AF0940EF66E87
:1015B000010EF76E000EF86EDA51F626000E086E78
:1015C000F7220850F8220900F55062EC02F0000101
:1015D000DA2B080EDA5DD8A4EFEF08F01200CB6F1B
:1015E000000ECA5DD8A401EF0BF0010EC95DD8A4AE
:1015F00001EF0BF0860EC85DD8A401EF0BF0A00E32
:10160000C75DD8B40EEF0BF0D8B00EEF0BF0200E84
:10161000CD6FCE6BCF6BD06B34EF0BF0A00E106E96
:10162000860E116E010E126E136AC751086EC851F4
:10163000096EC9510A6ECA510B6EFDEC00F01450D0
:101640000001D16F1550D26F1650D36F1750D46F61
:10165000300ED125CD6F000ED221CE6F000ED321DA
:10166000CF6F000ED421D06FCC510201286F000142
:10167000CB516AEC02F00001CD5166EC02F00001A2
:10168000CC2B000ECA5DD8A452EF0BF0000EC95D42
:10169000D8A452EF0BF0270EC85DD8A452EF0BF080
:1016A000100EC75DD8B45FEF0BF0D8B05FEF0BF052
:1016B000200ECD6FCE6BCF6BD06B9EEF0BF0A00EDC
:1016C000106E860E116E010E126E136AC751086EEF
:1016D000C851096EC9510A6ECA510B6EFDEC00F07B
:1016E0000C500001D16F0D50D26F0E50D36F0F50C0
:1016F000D46F100E106E270E116E126A136AD1513C
:10170000086ED251096ED3510A6ED4510B6EFDECA6
:1017100000F014500001D56F1550D66F1650D76FDA
:101720001750D86F300ED525CD6F000ED621CE6F55
:10173000000ED721CF6F000ED821D06FCC510201FF
:10174000286F0001CB516AEC02F00001CD5166EC2C
:1017500002F00001CC2B000ECA5DD8A4BCEF0BF048
:10176000000EC95DD8A4BCEF0BF0030EC85DD8A471
:10177000BCEF0BF0E80EC75DD8B4C9EF0BF0D8B0E2
:10178000C9EF0BF0200ECD6FCE6BCF6BD06B07EF98
:101790000CF0100E106E270E116E126A136AC751EC
:1017A000086EC851096EC9510A6ECA510B6EFDEC24
:1017B00000F00C500001D16F0D50D26F0E50D36F5E
:1017C0000F50D46FE80E106E030E116E126A136A7A
:1017D000D151086ED251096ED3510A6ED4510B6E9D
:1017E000FDEC00F014500001D56F1550D66F165067
:1017F000D76F1750D86F300ED525CD6F000ED6217C
:10180000CE6F000ED721CF6F000ED821D06FCC51F4
:101810000201286F0001CB516AEC02F00001CD51AA
:1018200066EC02F00001CC2B000ECA5DD8A425EFB7
:101830000CF0000EC95DD8A425EF0CF0000EC85DB9
:10184000D8A425EF0CF0640EC75DD8B432EF0CF0CD
:10185000D8B032EF0CF0200ECD6FCE6BCF6BD06BCB
:101860006FEF0CF0E80E106E030E116E126A136A21
:10187000C751086EC851096EC9510A6ECA510B6E24
:10188000FDEC00F00C500001D16F0D50D26F0E50E6
:10189000D36F0F50D46F640E106E116A126A136A00
:1018A000D151086ED251096ED3510A6ED4510B6ECC
:1018B000FDEC00F014500001D56F1550D66F165096
:1018C000D76F1750D86F300ED525CD6F000ED621AB
:1018D000CE6F000ED721CF6F000ED821D06FCC5124
:1018E0000201286F0001CB516AEC02F00001CD51DA
:1018F00066EC02F00001CC2B000ECA5DD8A48DEF7F
:101900000CF0000EC95DD8A48DEF0CF0000EC85D80
:10191000D8A48DEF0CF00A0EC75DD8B49AEF0CF086
:10192000D8B09AEF0CF0200ECD6FCE6BCF6BD06B92
:10193000D6EF0CF0640E106E116A126A136AC7516A
:10194000086EC851096EC9510A6ECA510B6EFDEC82
:1019500000F00C500001D16F0D50D26F0E50D36FBC
:101960000F50D46F0A0E106E116A126A136AD151A9
:10197000086ED251096ED3510A6ED4510B6EFDEC34
:1019800000F014500001D56F1550D66F1650D76F68
:101990001750D86F300ED525CD6F000ED621CE6FE3
:1019A000000ED721CF6F000ED821D06FCC5102018D
:1019B000286F0001CB516AEC02F00001CD5166ECBA
:1019C00002F00001CC2B0A0E106E116A126A136A23
:1019D000C751086EC851096EC9510A6ECA510B6EC3
:1019E000FDEC00F00C500001D16F0D50D26F0E5085
:1019F000D36F0F50D46F300ED125CD6F000ED22192
:101A0000CE6F000ED321CF6F000ED421D06FCC51FA
:101A10000201286F0001CB516AEC02F00001CD51A8
:101A200066EC02F00001CC2B12000F0E0201286FB1
:101A3000010E6AEC02F02A0E66EC02F0010E0201C1
:101A4000336F346BDCEC01F00F0E0201286F010ED6
:101A50006AEC02F0200E66EC02F0010E0201336F18
:101A6000346BDCEF01F0010E02011E6F1F6BC4EC42
:101A700002F0346E020E02011E6F1F6BC4EC02F006
:101A8000356E030E02011E6F1F6BC4EC02F0366E42
:101A9000040E02011E6F1F6BC4EC02F0416E426A1D
:101AA000050E02011E6F1F6BC4EC02F0406E060EA5
:101AB00002011E6F1F6BC4EC02F0376E070E0201AD
:101AC0001E6F1F6BC4EC02F0386E080E02011E6F11
:101AD0001F6BC4EC02F0396E090E02011E6F1F6B02
:101AE000C4EC02F03E6E3F6A0A0E02011E6F1F6BCD
:101AF000C4EC02F03A6E3B6A1E0E345C0001C391E6
:101B0000D8B485EF0DF0D8B0C381050E345CC39313
:101B1000D8B48DEF0DF0D8A0C383C395C3A1C3B3D0
:101B2000C385C3A596EF0DF00A0E346E1E0E355C0C
:101B3000C397D8B49EEF0DF0D8B0C387050E355CBF
:101B4000C399D8B4A6EF0DF0D8A0C389C39BC3A78F
:101B5000C3B9C38BC3ABAFEF0DF00A0E356EC80E21
:101B6000365CC39DD8B4B7EF0DF0D8B0C38D0A0E64
:101B7000365CC39FD8B4BFEF0DF0D8A0C38FC4911B
:101B8000C3ADC3BFC481C4A1C8EF0DF0320E366E21
:101B9000000E425CD8A4CFEF0DF0C80E415CC49398
:101BA000D8B4D5EF0DF0D8B0C483000E425CD8A4F1
:101BB000DCEF0DF00A0E415CC495D8B4E2EF0DF0F5
:101BC000D8A0C485C497C4A3C4B5C487C4A7ECEF88
:101BD0000DF0280E416E426AC80E405CC499D8B41C
:101BE000F4EF0DF0D8B0C4890A0E405CC49BD8B4A1
:101BF000FCEF0DF0D8A0C48BC49DC4A9C4BBC48D98
:101C0000C4AD05EF0EF01E0E406EC80E375CC49FCB
:101C1000D8B40DEF0EF0D8B0C48F0A0E375CC59162
:101C2000D8B415EF0EF0D8A0C581C593C4AFC5B127
:101C3000C583C5A31EEF0EF0550E376EC80E385C77
:101C4000C595D8B426EF0EF0D8B0C5850A0E385C1D
:101C5000C597D8B42EEF0EF0D8A0C587C599C5A5F5
:101C6000C5B7C589C5A937EF0EF09E0E386E1E0E9A
:101C7000395CC59BD8B43FEF0EF0D8B0C58B020ECF
:101C8000395CC59DD8B447EF0EF0D8A0C58DC59F6F
:101C9000C5ABC5BDC58FC5AF50EF0EF0050E396E93
:101CA000000E3F5CD8A457EF0EF0C80E3E5CC69104
:101CB000D8B45DEF0EF0D8B0C681000E3F5CD8A45A
:101CC00064EF0EF00A0E3E5CC693D8B46AEF0EF0D5
:101CD000D8A0C683C695C6A1C6B3C685C6A574EFEF
:101CE0000EF0460E3E6E3F6A000E3F5CD8A47BEFBE
:101CF0000EF0140E3E5CD8B484EF0EF0D8B084EF32
:101D00000EF0140E3E6E3F6A000E3B5CD8A48BEFC3
:101D10000EF0FA0E3A5CD8B494EF0EF0D8A094EF1F
:101D20000EF01E0E3A6E3B6A4150BB6F4250BC6FC4
:101D3000BD6BBE6B3850086E096ABB510A6EBC5150
:101D40000B6EBD510C6EBE510D6ECEEC00F00E5000
:101D50000001BF6F0F50C06F1050C16F1150C26FA4
:101D6000E80E106E030E116E126A136ABF51086EF0
:101D7000C051096EC1510A6EC2510B6EFDEC00F0EC
:101D80001450436E1550446E3E50106E3F50116E0D
:101D9000126A136AD00E086E120E096E130E0A6EC6
:101DA0000B6AFDEC00F014504B6E15504C6ED88051
:101DB000FF0E4B56FF0E4C561200F2A4E8EF0EF049
:101DC000302AD8B4312A4C50D76E4B50D66EF2948C
:101DD000110033EC0DF00001B96B1E50F3EC04F070
:101DE0001E6E0001F9511D6E1E5049EC01F0345079
:101DF00002013F6F406B94EC01F00001B92B0A0E19
:101E0000B95DD8A4EDEF0EF082A21BEF0FF0190E12
:101E1000D4EC08F0010E0201336F346BDCEC01F0FE
:101E2000010E7BEC02F0010E0201336F346BDCEC2F
:101E300001F004EF0FF082B230EF0FF01E50F3EC20
:101E400004F01E6E0001F9511D6E1E5049EC01F0A8
:101E5000345002013F6F406B94EC01F01BEF0FF028
:101E60000001BA6B1E503BEC05F01E6E0001F751ED
:101E70001D6E1E5049EC01F0345002013F6F406B63
:101E800094EC01F00001BA2B320EBA5DD8A432EF07
:101E90000FF0010E226E236A82B264EF0FF01E5023
:101EA0003BEC05F01E6E0001F7511D6E1E5049EC13
:101EB00001F0345002013F6F406B94EC01F0222A94
:101EC000D8B4232A4CEF0FF0030E0201396F3A6B9E
:101ED000B6EC01F022502E6E23502F6E608012005F
:101EE0000001B89182B2B881D88460A07DEF0FF074
:101EF000B8A17EEF0FF07FEF0FF0B8B1D894D8B44F
:101F0000B2EF0FF023502F5CD8A489EF0FF02250CE
:101F10002E5CD8B498EF0FF0D8B098EF0FF0D880BF
:101F200022502E543C6E23502F543D6E9FEF0FF0E5
:101F3000D8802E5022543C6E2F5023543D6E006AA0
:101F40003D50005CD8A4A7EF0FF03C50395CD8B4EA
:101F5000B2EF0FF0D8B0B2EF0FF0080ED4EC08F0EB
:101F6000E9EC0EF060900001B8B1608012008A8840
:101F70000A0E3602F3500001B76FB75102013F6FEE
:101F8000406B94EC01F082B4C3EF0FF08A980A0E14
:101F900002013F6F406B94EF01F082B4B7EC0FF099
:101FA0002250245C086E2350255C0810D8B42AEF18
:101FB00010F02350255CD8A4E0EF0FF02250245CF1
:101FC000D8B4FFEF0FF0D8A0FFEF0FF0060E2224D9
:101FD0000001B56F000E2320B66F255CD8A4F3EF87
:101FE0000FF0B551245CD8B4FDEF0FF0D8B0FDEF81
:101FF0000FF083EC06F0FFEF0FF083EC05F02350B9
:10200000255CD8A406EF10F02250245CD8B426EF4B
:1020100010F0D8B026EF10F0060E24240001B56FA2
:10202000000E2520B66F2350B65DD8A41AEF10F02D
:102030002250B55DD8B424EF10F0D8B024EF10F0E2
:10204000B5EC05F026EF10F0B5EC06F070EC0FF0F3
:10205000D0EF0FF0120082B4B7EC0FF026502A5CDC
:10206000086E27502B5C081228502C5C081229504F
:102070002D5C0810D8B4C0EF10F029502D5CD8A406
:102080004EEF10F028502C5CD8A44EEF10F02750E3
:102090002B5CD8A44EEF10F026502A5CD8B47DEF0C
:1020A00010F0D8A07DEF10F0060E26240001B16FCD
:1020B000000E2720B26F000E2820B36F000E2920DB
:1020C000B46F2D5CD8A471EF10F0B3512C5CD8A480
:1020D00071EF10F0B2512B5CD8A471EF10F0B15138
:1020E0002A5CD8B47BEF10F0D8B07BEF10F039EC5D
:1020F00007F07DEF10F039EC06F029502D5CD8A4E4
:102100008EEF10F028502C5CD8A48EEF10F02750E2
:102110002B5CD8A48EEF10F026502A5CD8B42EEF9A
:1021200010F0D8B02EEF10F0060E2A240001B16F87
:10213000000E2B20B26F000E2C20B36F000E2D204E
:10214000B46F2950B45DD8A4B2EF10F02850B35D3D
:10215000D8A4B2EF10F02750B25DD8A4B2EF10F0BF
:102160002650B15DD8B4BCEF10F0D8B0BCEF10F081
:10217000EAEC05F02EEF10F0EAEC06F02EEF10F08E
:1021800012000001A16FA1AFCBEF10F0476AF00E73
:10219000A115466E1200040E475CD8B4D4EF10F0BF
:1021A000D8B0D4EF10F0472A4704D8A4DAEF10F0E3
:1021B000A151486E020E475CAA95D8B4AA85140EA8
:1021C000485CAA97D8B4E7EF10F0D8B0AA87AA89DC
:1021D000AAB5AAA7AA99AAA96BEF11F0A151496EB5
:1021E0004850AB6FAC6BAB5102011E6F0001AC519C
:1021F00002011F6FC4EC02F00001AD6FA46FA26F6B
:10220000800E4824A46FAE6FAF6BAE5102011E6FFB
:102210000001AF5102011F6FC4EC02F00001B06F6A
:10222000A46FA36F900E465CD8A42FEF11F0495015
:10223000A46FA56BA551A76FA405A66FA629D8B456
:10224000A707780EA603F350A86FF450A96F780E75
:10225000A703F350A927A851A227A951A323800EB1
:10226000465CD8A442EF11F0A2514924A46F000E9D
:10227000086EA3510820A56FA36FA405A26FA22921
:10228000D8B4A30748500201166F176B0001A25182
:10229000D5EC02F0800E48240001A46F0201166FF5
:1022A000176B0001A351D5EC02F048500001C76F35
:1022B000C86BC96BCA6BCC6B010EEFEC0AF0000166
:1022C000A251C76FA351C86FC96BCA6B090ECC6FFF
:1022D000010EEFEF0AF0120000019C6F9CAF79EF46
:1022E00011F0476AF00E9C15466E0F0E9C159D6FFF
:1022F0001200040E475CD8B482EF11F0D8B082EF20
:1023000011F0472A4704D8A488EF11F09C51486E79
:10231000020E475CD8A430EF12F09C51496E495030
:10232000D8A495EF11F0800E466E9D51455CD8A45F
:1023300030EF12F0900E465CD8A4ABEF11F0D890BD
:1023400048349E6F01EE00F09E51E9263050EF6E4A
:10235000E92A3150EF6E800E465CD8A4E4EF11F00C
:1023600030504F6E3150506ED89048349E6F01EE11
:1023700000F09E51E926EF504D6EE92AEF504E6E67
:10238000D89048349E6F01EE00F09E51E926EF6A26
:10239000E92AEF6A4D504E10D8B4E4EF11F04850DE
:1023A000B4EC03F04850B4EC03F04D50B4EC03F03F
:1023B0004E50B4EC03F04F50B4EC03F05050B4EC7A
:1023C00003F0322AD8B4332AB00E465CD8A430EFDA
:1023D00012F030504F6E3150506E486A0001A06BC1
:1023E000D89048349E6F01EE00F09E51E926EF50E0
:1023F000E92AEF10D8B428EF12F0D89048349F6F34
:1024000001EE00F09F51E926EF504D6EE92AEF50A2
:102410004E6ED89048349E6F01EE00F09E51E92632
:10242000EF6AE92AEF6A4850B4EC03F04850B4EC84
:1024300003F04D50B4EC03F04E50B4EC03F04F50A9
:10244000B4EC03F05050B4EC03F0322AD8B4332A81
:10245000482A0001A02B800EA05DD8A4F0EF11F057
:10246000120033EC0DF0050E0201396F3A6BB6EC39
:1024700001F080B64DEF12F01C0ED4EC08F080A6EF
:102480003FEF12F0020E0201336F346BDCEC01F00F
:1024900080A64DEF12F048EF12F080B254EF12F028
:1024A00015EC0DF0C0EF13F0060E3202F3500001F0
:1024B0008A6FF4508B6F060E3302F3508B278A51CC
:1024C0000201006F00018B510201016F026B036B6F
:1024D000BAEC03F0FAEC03F00001886FFAEC03F0B9
:1024E000486EFAEC03F04D6EFAEC03F04E6EFAEC27
:1024F00003F04F6EFAEC03F0506EFFEC03F048501F
:102500000001C76FC86BC96BCA6BCC6B010EEFECD7
:102510000AF032500001C76F3350C86FC96BCA6BE5
:10252000090ECC6F010EEFEC0AF0322AD8B4332A30
:10253000C80E485CD8B4C0EF13F0800E485C0001B0
:10254000929BD8B4A6EF12F0D8B0928B4850885D19
:10255000929DD8A4928D929F92AB92BD928F92AF92
:10256000BAEF12F01D0ED4EC08F080A2C0EF13F009
:10257000B5EF12F0130E485CD8B439EF12F0D8A0C2
:1025800039EF12F04850946F956B945102011E6F11
:102590000001955102011F6FC4EC02F00001966F1B
:1025A0008A6F206E800E48248A6F976F986B9751C0
:1025B00002011E6F0001985102011F6FC4EC02F06E
:1025C0000001996F8A6F216E20502110D8B439EF25
:1025D00012F02050246E2150256ECDEC0FF0D880E3
:1025E0004F504D54516E50504E54526E0A0E51027F
:1025F000F35000018A6FF4508B6F0A0E5202F350B1
:102600008B27D8808A514054516E000E086E8B5132
:102610000854526ED89042308B6F41308A6F5150BF
:102620008A258C6F52508B218D6F4150106E425015
:10263000116E126A136A8C51086E8D51096E0A6A06
:102640000B6AFDEC00F014500001896F51508A6F45
:1026500052508B6F8C6B8D6B3850086E096A8A51A3
:102660000A6E8B510B6E8C510C6E8D510D6ECEEC33
:1026700000F00E5000018E6F0F508F6F1050906F52
:102680001150916F640E106E116A126A136A8E51A6
:10269000086E8F51096E90510A6E91510B6EFDECD0
:1026A00000F01450516E1550526E00018951106E99
:1026B000116A126A136A5150086E5250096E0A6A02
:1026C0000B6AFDEC00F01450436E1550446E4D50F3
:1026D00000018A6F4E508B6F8C6B8D6B3850086E7B
:1026E000096A8A510A6E8B510B6E8C510C6E8D519A
:1026F0000D6ECEEC00F00E5000018E6F0F508F6FFC
:102700001050906F1150916F0A0E106E116A126A7C
:10271000136A8E51086E8F51096E90510A6E915155
:102720000B6EFDEC00F014502A6E15502B6E1650F7
:102730002C6E17502D6E2BEC10F0B7EC0FF0000143
:1027400089519A6F9B6BB9EF13F0265043242A6E80
:10275000275044202B6E000E086E285008202C6E47
:10276000295008202D6E2BEC10F0B7EC0FF0000173
:102770009B2B9B519A5DD8A4A5EF13F039EF12F073
:1027800032063228D8B43306100E0201166F176BCA
:102790003250D5EC02F0110E0201166F176B335058
:1027A000D5EF02F00A0ED4EC08F0140E486E0001CA
:1027B000876B48500201166F176B000ED5EC02F0C4
:1027C000482A0001872BEC0E875DD8A4D9EF13F0BF
:1027D0000B0ED4EC08F0010E0201336F346BDCEF0A
:1027E00001F0000E7BEC02F0010E7BEC02F0000128
:1027F000DC6B140E83EC07F0020E0201336F346BB6
:10280000DCEC01F033EC0DF082B4B7EC0FF0150EF8
:10281000D4EC08F0E9EC0EF0140ED4EC08F0010E44
:10282000246E256ACDEC0FF02A6A2B6A2C6A2D6A79
:10283000010E536E0001DC6B000E83EC07F0010EFD
:102840000201336F346BDCEC01F0010E7BEC02F023
:1028500082A059EF14F080B43BEF14F0010E535CEA
:10286000D8B439EF14F0D8A039EF14F053063BEF89
:1028700014F00C0E536E80B84BEF14F00C0E535C3A
:10288000D8B449EF14F0D8B049EF14F0532A4BEF05
:1028900014F0010E536E010E0001DC6F535083ECF7
:1028A00007F0010E0201336F346BDCEC01F028EF0E
:1028B00014F033EC0DF05304D8A400EF15F0010E22
:1028C0007BEC02F00001DC6B010E83EC07F0010EE3
:1028D0000201336F346BDCEC01F080A200EF15F0E5
:1028E00080B87DEF14F0010E2224246E000ED8B0C3
:1028F000010E2324256ECDEC0FF080B496EF14F07A
:10290000000E235CD8A487EF14F0010E225CD8B42B
:1029100096EF14F0D8A096EF14F02350256E220401
:10292000246E2428D8B42506CDEC0FF084B0ADEF8A
:1029300014F0010E26242A6E000ED8B0010E2724B2
:102940002B6E000ED8B0010E28242C6E000ED8B0CD
:10295000010E29242D6E2BEC10F080B0D9EF14F06D
:10296000000E295CD8A4C1EF14F0000E285CD8A496
:10297000C1EF14F0000E275CD8A4C1EF14F0010ED3
:10298000265CD8B4D9EF14F0D8A0D9EF14F02950B0
:102990002D6E28502C6E27502B6E010E265C2A6E51
:1029A000010ED8A02B5ED8A02C5ED8A02D5E2BECFB
:1029B00010F080B6E4EF14F0B7EC0FF0050E020152
:1029C000396F3A6BB6EC01F022500001C76F23500B
:1029D000C86FC96BCA6B020ECC6F010EEFEC0AF028
:1029E00026500001C76F2750C86F2850C96F295063
:1029F000CA6F090ECC6F010EEFEC0AF06DEF14F008
:102A0000020E535CD8A463EF15F0486A716AD8903F
:102A10004834546E01EE00F05450E926EF6AE92A7A
:102A2000EF6A482A712A800E715CD8A407EF15F06E
:102A3000326A336A010E7BEC02F00001DC6B020E9D
:102A400083EC07F0010E0201336F346BDCEC01F014
:102A5000306A316AF294D58E0201076B086B096BFC
:102A60000A6B78EC03F01B0ED4EC08F015EC03F0C5
:102A70004A6E629408B0628462A442EF15F04A5034
:102A80006CEC11F080B236EF15F0726AC80EB4EC3F
:102A900003F0722A1E0E725CD8A446EF15F0B8EC53
:102AA00003F0D59E32500001C76F3350C86FC96B19
:102AB000CA6BCC6B010EEFEC0AF0020E0201336F11
:102AC000346BDCEC01F0030E535CD8A47EEF15F000
:102AD000326A336A266A276A286A296A010E7BEC01
:102AE00002F00001DC6B030E83EC07F0010E020123
:102AF000336F346BDCEC01F031EC12F0040E535CFC
:102B0000D8A476EF16F0010E7BEC02F00001DC6B2E
:102B1000040E83EC07F0010E0201336F346BDCEC22
:102B200001F0100E02011E6F1F6BC4EC02F0326E3A
:102B3000110E02011E6F1F6BC4EC02F0336E060E05
:102B40003202F350546EF450556E060E3302F350B9
:102B5000552654500201006F5550016F026B036BF4
:102B6000BAEC03F0FAEC03F0486EFAEC03F0486EAE
:102B7000FAEC03F04D6EFAEC03F04E6EFAEC03F053
:102B80004F6EFAEC03F0506EFFEC03F0485000017A
:102B9000C76FC86BC96BCA6BCC6B010EEFEC0AF048
:102BA00032500001C76F3350C86FC96BCA6B090E32
:102BB000CC6F010EEFEC0AF082A042EF16F06390AA
:102BC00080A86380639280A46382639463A063B2ED
:102BD000638463A4DCEF15F080B4FAEF15F0325093
:102BE0003310D8B4FDEF15F032063228D8B43306CE
:102BF000FDEF15F0322AD8B4332A060E3202F35014
:102C0000546EF450556E060E3302F3505526545050
:102C10000201006F5550016F026B036BBAEC03F0B9
:102C2000FAEC03F0486EFAEC03F0486EFAEC03F0AD
:102C30004D6EFAEC03F04E6EFAEC03F04F6EFAECC8
:102C400003F0506EFFEC03F048500001C76FC86BF3
:102C5000C96BCA6BCC6B010EEFEC0AF0325000016D
:102C6000C76F3350C86FC96BCA6B090ECC6F010EAA
:102C7000EFEC0AF0010E0201336F346BDCEC01F073
:102C8000DCEF15F04D50546E4E50556E566A576A33
:102C90003850086E096A54500A6E55500B6E5650E3
:102CA0000C6E57500D6ECEEC00F00E50586E0F505B
:102CB000596E10505A6E11505B6E0A0E106E116AEA
:102CC000126A136A5850086E5950096E5A500A6EAB
:102CD0005B500B6EFDEC00F01450266E1550276E05
:102CE0001650286E1750296E31EC12F0050E535C09
:102CF000D8A4B2EF19F0010E7BEC02F00001DC6BFE
:102D0000050E83EC07F0010E0201336F346BDCEC2F
:102D100001F0010ED4EC08F034500001C76FC86B0D
:102D2000C96BCA6B090ECC6F010EEFEC0AF0010EF5
:102D30000201336F346BDCEC01F080A2DCEF16F0A3
:102D400080A8342A80A434061E0E345C6492D8B461
:102D5000ACEF16F0D8B06482050E345C6494D8B43D
:102D6000B4EF16F0D8A06484649664A264B4648658
:102D700064A6BDEF16F00A0E346E34500001C76F22
:102D8000C86BC96BCA6B090ECC6F010EEFEC0AF071
:102D9000010E0201336F346BDCEC01F082B09DEF69
:102DA00016F0010E0201166F176B3450D5EC02F0CD
:102DB00015EC0DF09DEF16F0010E0201336F346B30
:102DC000DCEC01F0020ED4EC08F035500001C76FC6
:102DD000C86BC96BCA6B090ECC6F010EEFEC0AF021
:102DE000010E0201336F346BDCEC01F080A235EF91
:102DF00017F080A8352A80A435061E0E355C659034
:102E0000D8B405EF17F0D8B06580050E355C659233
:102E1000D8B40DEF17F0D8A06582659465A065B2AF
:102E2000658465A416EF17F00A0E356E3550000163
:102E3000C76FC86BC96BCA6B090ECC6F010EEFEC84
:102E40000AF0010E0201336F346BDCEC01F082B04A
:102E5000F6EF16F0020E0201166F176B3550D5EC27
:102E600002F015EC0DF0F6EF16F0010E0201336FD3
:102E7000346BDCEC01F0030ED4EC08F036500001AA
:102E8000C76FC86BC96BCA6B090ECC6F010EEFEC34
:102E90000AF0010E0201336F346BDCEC01F080A20A
:102EA0008EEF17F080A8362A80A43606C80E365C4E
:102EB000659ED8B45EEF17F0D8B0658E0A0E365C0A
:102EC0006690D8B466EF17F0D8A06680669265AEBB
:102ED00066B0668266A26FEF17F01E0E366E365031
:102EE0000001C76FC86BC96BCA6B090ECC6F010EAE
:102EF000EFEC0AF0010E0201336F346BDCEC01F0F1
:102F000082B04FEF17F0030E0201166F176B3650A9
:102F1000D5EC02F015EC0DF04FEF17F0010E0201A9
:102F2000336F346BDCEC01F0040ED4EC08F041504C
:102F30000001C76F4250C86FC96BCA6B090ECC6FD6
:102F4000010EEFEC0AF0010E0201336F346BDCEC82
:102F500001F080A2FDEF17F080B8B2EF17F0412A20
:102F6000D8B4422A80B4B9EF17F041064128D8B44A
:102F70004206000E425CD8A4C0EF17F0C80E415CB8
:102F8000669CD8B4C6EF17F0D8B0668C000E425CD1
:102F9000D8A4CDEF17F00A0E415C669ED8B4D3EFEB
:102FA00017F0D8A0668E679066AC66BE678067A093
:102FB000DDEF17F0140E416E426A41500001C76FF9
:102FC0004250C86FC96BCA6B090ECC6F010EEFEC93
:102FD0000AF0010E0201336F346BDCEC01F082B0B9
:102FE000A9EF17F0040E0201166F176B4150D5ECD4
:102FF00002F015EC0DF0A9EF17F0010E0201336F8E
:10300000346BDCEC01F0050ED4EC08F0405000010C
:10301000C76FC86BC96BCA6B090ECC6F010EEFECA2
:103020000AF0010E0201336F346BDCEC01F080A278
:1030300056EF18F080A8402A80A44006C80E405CD5
:10304000679AD8B426EF18F0D8B0678A0A0E405CA9
:10305000679CD8B42EEF18F0D8A0678C679E67AA3B
:1030600067BC678E67AE37EF18F01E0E406E40509B
:103070000001C76FC86BC96BCA6B090ECC6F010E1C
:10308000EFEC0AF0010E0201336F346BDCEC01F05F
:1030900082B017EF18F0050E0201166F176B405043
:1030A000D5EC02F015EC0DF017EF18F0010E02014F
:1030B000336F346BDCEC01F0060ED4EC08F03750C3
:1030C0000001C76FC86BC96BCA6B090ECC6F010ECC
:1030D000EFEC0AF0010E0201336F346BDCEC01F00F
:1030E00080A2AFEF18F080A8372A80A43706E60E3A
:1030F000375C6898D8B47FEF18F0D8B068880A0EAB
:10310000375C689AD8B487EF18F0D8A0688A689CB2
:1031100068A868BA688C68AC90EF18F0640E376ED7
:1031200037500001C76FC86BC96BCA6B090ECC6FF3
:10313000010EEFEC0AF0010E0201336F346BDCEC90
:1031400001F082B070EF18F0060E0201166F176BD7
:103150003750D5EC02F015EC0DF070EF18F0010EC1
:103160000201336F346BDCEC01F0070ED4EC08F095
:1031700038500001C76FC86BC96BCA6B090ECC6FA2
:10318000010EEFEC0AF0010E0201336F346BDCEC40
:1031900001F080A208EF19F080A8382A80A4380630
:1031A000E60E385C6996D8B4D8EF18F0D8B06986C6
:1031B0000A0E385C6998D8B4E0EF18F0D8A0698896
:1031C000699A69A669B8698A69AAE9EF18F0640E74
:1031D000386E38500001C76FC86BC96BCA6B090ED7
:1031E000CC6F010EEFEC0AF0010E0201336F346B6D
:1031F000DCEC01F082B0C9EF18F0070E0201166F87
:10320000176B3850D5EC02F015EC0DF0C9EF18F043
:10321000010E0201336F346BDCEC01F0080ED4ECCC
:1032200008F039500001C76FC86BC96BCA6B090E33
:10323000CC6F010EEFEC0AF0010E0201336F346B1C
:10324000DCEC01F080A261EF19F080A8392A80A49B
:1032500039061E0E395C6A94D8B431EF19F0D8B033
:103260006A84020E395C6A96D8B439EF19F0D8A096
:103270006A866A986AA46AB66A886AA842EF19F0F0
:10328000050E396E39500001C76FC86BC96BCA6B28
:10329000090ECC6F010EEFEC0AF0010E0201336F44
:1032A000346BDCEC01F082B022EF19F0080E020161
:1032B000166F176B3950D5EC02F015EC0DF022EFBC
:1032C00019F0010E0201336F346BDCEC01F00C0ECF
:1032D000D4EC08F03A500001C76F3B50C86FC96B7F
:1032E000CA6B090ECC6F010EEFEC0AF0010E020161
:1032F000336F346BDCEC01F080A2ACEF19F080B8D6
:1033000085EF19F03A2AD8B43B2A80B48CEF19F033
:103310003A063A28D8B43B063A500001C76F3B50F2
:10332000C86FC96BCA6B090ECC6F010EEFEC0AF0C7
:10333000010E0201336F346BDCEC01F082B07CEFE4
:1033400019F0090E0201166F176B3A50D5EC02F016
:1033500015EC0DF07CEF19F0010E0201336F346BA8
:10336000DCEC01F0060E535CD8A4E4EF1AF0010E79
:103370007BEC02F00001DC6B060E83EC07F0010E23
:103380000201336F346BDCEC01F0140E486E80A246
:10339000DEEF1AF04850736E746A735002011E6FAC
:1033A00074501F6FC4EC02F0756E546E206E800E68
:1033B0004824546E766E776A765002011E6F7750FD
:1033C0001F6FC4EC02F0786E546E216E2050000125
:1033D000C76F2150C86FC96BCA6B0A0ECC6F000E45
:1033E000EFEC0AF022500001C76F2350C86FC96B81
:1033F000CA6B010ECC6F010EEFEC0AF048500001D1
:10340000C76FC86BC96BCA6B090ECC6F010EEFECAE
:103410000AF06B9880A06B886B9A84A06B8A6B9C77
:103420006BA86BBA6B8C6BAC37EF1AF080B01CEFEB
:103430001AF0482A1DEF1AF04806140E485CD8B45A
:1034400027EF1AF0D8B027EF1AF07F0E486E7F0EE4
:10345000485CD8B431EF1AF0D8A031EF1AF0140E4E
:10346000486E050E0201396F3A6BB6EC01F080B878
:1034700044EF1AF0010E2224246E000ED8B0010E83
:103480002324256ECDEC0FF080B45DEF1AF0000E12
:10349000235CD8A44EEF1AF0010E225CD8B45DEF85
:1034A0001AF0D8A05DEF1AF02350256E2204246E86
:1034B0002428D8B42506CDEC0FF080B6A0EF1AF082
:1034C0003A50546E3B50556E566A576A3750086EE4
:1034D000096A54500A6E55500B6E56500C6E575078
:1034E0000D6ECEEC00F00E50586E0F50596E10500D
:1034F0005A6E11505B6E640E106E116A126A136A76
:103500005850086E5950096E5A500A6E5B500B6E37
:10351000FDEC00F014505C6E15505D6E16505E6E42
:1035200017505F6E22505C24246E23505D20256E60
:10353000CDEC0FF0050E0201396F3A6BB6EC01F0DD
:1035400082B0D6EF1AF022042310D8A4AAEF1AF002
:10355000226A236A48500201166F176B2250D5EC7D
:1035600002F0800E4824546E0201166F176B235030
:10357000D5EC02F022500001C76F2350C86FC96B11
:10358000CA6B0A0ECC6F000EEFEC0AF015EC0DF0D2
:1035900022502310D8A4D0EF1AF0010E226E236A15
:1035A000050E0201396F3A6BB6EC01F0010E020113
:1035B000396F3A6BB6EC01F0C7EF19F0010E02015A
:1035C000336F346BDCEC01F0070E535CD8A45AEF78
:1035D0001BF0010E7BEC02F00001DC6B070E83ECAC
:1035E00007F0010E0201336F346BDCEC01F0090EC1
:1035F000D4EC08F0010E0201336F346BDCEC01F007
:1036000080A254EF1BF080B809EF1BF03E2AD8B41B
:103610003F2A80B410EF1BF03E063E28D8B43F0688
:10362000000E3F5CD8A417EF1BF0C80E3E5C6D9AED
:10363000D8B41DEF1BF0D8B06D8A000E3F5CD8A443
:1036400024EF1BF0140E3E5C6D9CD8B42AEF1BF0E7
:10365000D8A06D8C6D9E6DAA6DBC6D8E6DAE34EF75
:103660001BF0140E3E6E3F6A3E500001C76F3F5084
:10367000C86FC96BCA6B090ECC6F010EEFEC0AF074
:10368000050E0201396F3A6BB6EC01F082B000EF23
:103690001BF0090E0201166F176B3E50D5EC02F0BD
:1036A00015EC0DF000EF1BF0010E0201336F346BCF
:1036B000DCEC01F0080E535CD8A477EF1BF0010E90
:1036C0007BEC02F00001DC6B080E83EC07F0010ECE
:1036D0000201336F346BDCEC01F080A277EF1BF05A
:1036E00082B06DEF1BF0D2EC13F06DEF1BF0090E02
:1036F000535CD8A496EF1BF0010E7BEC02F00001A6
:10370000DC6B090E83EC07F0010E0201336F346BA2
:10371000DCEC01F080A296EF1BF082B08AEF1BF088
:1037200015EC0DF0E9EC0EF08AEF1BF00A0E535C7D
:10373000D8A436EF1CF0010E7BEC02F00001DC6B2C
:103740000A0E83EC07F0010E0201336F346BDCECE0
:1037500001F080A236EF1CF082B0A9EF1BF0140E2E
:10376000486E796A48500001C76FC86BC96BCA6B55
:10377000CC6B010EEFEC0AF048507A6E7B6A7A50FF
:1037800002011E6F7B501F6FC4EC02F07C6E546E02
:10379000206E800E4824546E7D6E7E6A7D5002013C
:1037A0001E6F7E501F6FC4EC02F07F6E546E216E50
:1037B00020502110D8B42DEF1CF0900E0DEC03F02A
:1037C00048500DEC03F0780E106E116A126A136AFD
:1037D0002050086E2150096E0A6A0B6AFDEC00F059
:1037E0001450546E1550556E010E5424566E000E32
:1037F000D8B0010E5524576E56500DEC03F0020E52
:103800000201396F3A6BB6EC01F0800E0DEC03F05B
:1038100048500DEC03F0780E106E116A126A136AAC
:103820002050086E2150096E0A6A0B6AFDEC00F008
:103830000C50546E0D50556E010E5424566E000EF1
:10384000D8B0010E5524576E56500DEC03F0020E01
:103850000201396F3A6BB6EC01F0482A792A6C0EF6
:10386000795CD8A4B2EF1BF0A9EF1BF00B0E535CF0
:10387000D8A468EF1CF0010E7BEC02F00001DC6BB9
:103880000B0E83EC07F0010E0201336F346BDCEC9E
:1038900001F0D2EC13F0010E7BEC02F080A268EF95
:1038A0001CF082B04EEF1CF01B0ED4EC08F015ECAF
:1038B00003F04A6E6F9E08B06F8E6FAE63EF1CF020
:1038C0004A50C1EC10F080B257EF1CF04EEF1CF0E4
:1038D0000C0E535CD8A418EF14F033EC0DF0010E6D
:1038E0007BEC02F00001DC6B0C0E83EC07F0010EA8
:1038F0000201336F346BDCEC01F0140E486E0001F2
:10390000806B050E0201396F3A6BB6EC01F080A2B4
:1039100018EF14F048500001816F826B8151020151
:103920001E6F0001825102011F6FC4EC02F0000102
:10393000836F546E206E800E4824546E846F856BA6
:10394000845102011E6F0001855102011F6FC4ECFA
:1039500002F00001866F546E216E4850C76FC86B2D
:10396000C96BCA6BCC6B010EEFEC0AF02050000162
:10397000C76F2150C86FC96BCA6B090ECC6F010E9F
:10398000EFEC0AF020502110D8B4D5EF1CF02050F5
:10399000246E2150256ECDEC0FF080B6CDEF1CF0DB
:1039A00080A218EF14F0B7EC0FF0482A0001802B2A
:0E39B0006C0E805DD8A481EF1CF018EF14F0AF
:020000040030CA
:0E0000000002191E008381000FC00FE00F40A8
:00000001FF
